:0300000002492F83
:0C492F0078FFE4F6D8FD75816E02497631
:10283E0020000A3C2E2E2E3E004950436F6E6E65D0
:10284E0063745245510A004950436F6E6E6563744E
:10285E00000A49504E6F41434B210A003E432C560D
:10286E002C43432CC0E4E0EFF2E5F020D1E8EDEA92
:10287E00EEEC49500A003E432C4D41432C2530329C
:10288E0062583A25303262583A25303262583A252B
:10289E00303262583A25303262583A253032625818
:1028AE002C4D414320E0E4F0E5F10A003E432C5666
:1028BE0045522C20332E3220EEF220257320257324
:1028CE002CC2E5F0F1E8FF20495020ECEEE4F3EBEA
:1028DE00FF0A00417567203132203230313000312D
:1028EE00353A31323A3333003E432C4C442C50525D
:1028FE004F473A202020202020202020202020205A
:10290E0020202020202020202020202020202020B9
:10291E0020202020202020202020202020202020A9
:10292E002020202020202020202020202020202099
:10293E0020202020202020202CC4E0F2E020EFF0E8
:10294E00EEF8E8E2EAE828F4E0E9EB290A003E2A8C
:10295E002C312CCEF1EDEEE2EDFBE520EFE0F0E0D8
:10296E00ECE5F2F0FB20F1E5F2E5E2EEE3EE20E835
:10297E00EDF2E5F0F4E5E9F1E00A003E412C4130DC
:10298E00312C2562752E2562752E2562752E2562D7
:10299E00752C495020E0E4F0E5F120E0E4E0EFF2A0
:1029AE00E5F0E00A003E412C4130322C2562752EB6
:1029BE002562752E2562752E2562752C495020E0F4
:1029CE00E4F0E5F120EEF1ED2E20F1E5F0E2E5F098
:1029DE00E00A003E412C4130332C2562752E2562D3
:1029EE00752E2562752E2562752C495020E0E4F077
:1029FE00E5F120F0E5E72E20F1E5F0E2E5F0E00A62
:102A0E00003E412C4130342C2562752E2562752EE8
:102A1E002562752E2562752CCCE0F1EAE020F1E5F9
:102A2E00F2E80A003E412C4130352C2562752E25E8
:102A3E0062752E2562752E2562752CD8EBFEE70A7F
:102A4E00003E2A2C312CC4EEEF2E20EFE0F0E0EC0D
:102A5E00E5F2F0FB20F1E5F2E5E2EEE3EE20E8ED43
:102A6E00F2E5F0F4E5E9F1E00A003E422C53303194
:102A7E002C2562752CC6E4E0F2FC20E7E0EFF0EEC8
:102A8E00F1E020F1EEE5E4E8EDE5EDE8FF20EEF211
:102A9E0020F1E5F0E2E5F0E00A003E422C53303240
:102AAE002C2562752CCEE1ECE5ED20F120F1E5F060
:102ABE00E2E5F0EEEC20E1E5E720EAE2E8F2E0ED17
:102ACE00F6E8E90A003E422C5330332C2562752C71
:102ADE00CFE5F0E5E7E0EFF3F1EA20EFF0E820EFE5
:102AEE00EEF2E5F0E520F1E2FFE7E820F120F1E576
:102AFE00F0E2E5F0EEEC0A003E422C5330382C2585
:102B0E0062752CCCE5E4EBE5EDEDFBE920495020B8
:102B1E00EAE0EDE0EB28E7E0E4E5F0E6EAE020E4C9
:102B2E00EE203520F1E5EA290A003E454E440A0022
:102B3E000A44756D7058202020202030302030310E
:102B4E0020303220303320303420303520303620C3
:102B5E00303720303820303920304120304220307C
:102B6E0043203044203045203046000A3A003A20B7
:102B7E00000A000A44756D70442020202020303059
:102B8E002030312030322030332030342030352088
:102B9E003036203037203038203039203041203048
:102BAE0042203043203044203045203046004572CC
:102BBE0072206B657900526420656570726F6D0AC4
:102BCE00005264204D454D0A00526420436F6465E7
:102BDE000A00577269746520436F64650A00446584
:102BEE006275674950204F4E0A0044656275674909
:102BFE0050204F46460A00446562756755736572EC
:102C0E00204F6E0A00446562756755736572204FDA
:102C1E0046460A0044656275674D7367204F6E0A1B
:102C2E000044656275674D7367204F46460A004340
:102C3E006F6E666967206C6F636B210A0057722096
:102C4E00656570726F6D0A0020536176652065654B
:102C5E0070726F6D210A00457272204D4143210042
:102C6E004C6F61643E3E002A00CEF8E8E1EAE00ACD
:102C7E0000202D202575282575290A003C4130316C
:102C8E003D003C4130323D003C4130333D003C4143
:102C9E0030343D003C4130353D003C21003C53304A
:102CAE00313D003C5330323D003C5330333D003C0F
:102CBE005330353D003C5330383D003C5330363DAB
:012CCE000005
:06529400010B00010900FE
:10528400C28E438910758BFF758DB7D2ABD28E2237
:03001B0002489FF9
:10489F00C0E0C083C082C0D0C28E758BFF758DB74C
:1048AF0020060675A61E75A6E10509D202E50B6066
:1048BF0002050B050EE50E540F7051E50AD3940156
:1048CF004002150AD20EE50E543F7012D2009066C8
:1048DF008EE0600A04F0E0D394B44002D2069066F2
:1048EF0087E0600204F0906104E0600214F09066CB
:1048FF008FE0D394014003E014F0300502050CE57E
:10490F000DD394644004D2068002050DE508D394BC
:10491F000140021508D28ED0D0D082D083D0E032A1
:101C3900C291C290D2B5C20B7D027C007F071252BD
:101C49004D8F50E550646060097D017F601251C875
:101C5900D20BE4FDFC7F0B12524D8F50E55030E65C
:101C6900097D04E4FF1251ECD20B7D017C007F0752
:101C790012524D8F50E5507008FD7FFF1251C8D2A6
:101C89000B300B03126000C288C2A8C2AA75890072
:101C9900124CD790633FE0B4FA06A3E064CE607BB0
:101CA900E4F55074372550F582E43463F583E4F0A4
:101CB9000550E550B443EC90633F74FAF0A374CE39
:101CC900F0A374CCF0906345740AF0E4A3F0A30484
:101CD900F0A3F090633B74FFF0A3F0A3F0E4A3F04A
:101CE9009063567403F0E4F550E5502401FFE433A2
:101CF900FE74372550F582E43463F583E0FD125113
:101D0900A40550E550C3944340DFE4F5A775A61E2A
:101D190075A6E1907FF0F0A3F080FE90634A74030A
:101D2900F0A374CCF0E4906349F090668CF0A3F0D2
:101D3900124341C2B512476FC20612502BD20BC2D1
:101D49000DC20C9065777408F09062B57424F0E4C4
:101D5900A3F090633FE09062B7F0906340E0906237
:101D6900B8F0906341E09062B9F0906342E090620C
:101D7900BAF0906343E09062BBF0906344E09062F4
:101D8900BCF0750A01E4906578F0C207C208C2097F
:101D9900C20A200B18AF50FE7D03124427E4FF123C
:101DA90046BF7E287F3EE4FBFDFC123F5E90668EB7
:101DB900E060037401F0E4906104F0F50C9065763D
:101DC900F0F50D12528475A70775A61E75A6E1D206
:101DD900AFE4F50D906104E0700312138D90668FE6
:101DE900E06401701D9080007410F09080A874FF69
:101DF900F0A3F0A3F0A3F0E490668FF0D20BC20C2D
:101E0900C20D908008E0F55030E405D2077410F057
:101E1900E55030E508D2099080087420F0E550308B
:101E2900E608D2089080087440F0E50CC39403409A
:101E390019908002E4F0908001F0908000F0E50CA8
:101E490094064006E4F50C12502B9080A0E0700334
:101E5900124E419080B8E07003124D559080D0E049
:101E69007003124FCF908000E070133007101240BA
:101E790065906332EFF0D394004003120AD4908046
:101E890002E07006908000E06005D205021DDAC20A
:101E990005E4F50C906104E06003021DDA200B12E1
:101EA900906579E0600C7E287F40124259E4906584
:101EB90079F0300912123BBB906332EFF0D39400F2
:101EC9004005E0FF12002220080302205E123A3486
:101ED900906332EFF07003021DDA906376E054BF2D
:101EE900247F7003021FB9147003021F912402603A
:101EF90003022000200B077E287F47124259200F3A
:101F09000302205E90634EE07006906352E06067C2
:101F1900906683E0FF90634EE0B50724906684E005
:101F2900FE90634FE0B50618906685E0FE90635019
:101F3900E0B5060C906686E0FE906351E06E60376E
:101F4900906352E06F600302205E906684E0FF9028
:101F59006353E06F600302205E906685E0FF906343
:101F690054E06F600302205E906686E0FF9063553F
:101F7900E06F600302205EC2039065787401F0127D
:101F8900529D750A0102205E90668EE0600374011D
:101F9900F090667BE0FF906378E06F600302205E5B
:101FA90090667BE004F0E4F50A906576F002205E25
:101FB90030030302205E906345E07003021DDA904E
:101FC90062B4E06008906356741EF0800690635610
:101FD9007403F012529CD203E4F50A906576F090EE
:101FE900668704F0E490667AF0A3F0200B677E28F8
:101FF9007F55124259805E90668EE060037401F04D
:10200900300352906376E020E74B906378E0FF90CD
:10201900667AE0FE6F600D906682E07007EE146FDD
:102029007033801390667AE004F0906332E0FFD356
:10203900940440031252109060007482F0A374015A
:10204900F0906378E0906002F07E607F007D03127B
:102059004A42021DDA20030302217CE50A706E124E
:102069003D2CEF60237E647F76906477E02404FD45
:10207900124A42906682E07009906356E0F50A02BE
:102089001DDAE4F50A021DDA906687E0D3943C4034
:102099003C906682E070369062B4E070309066875A
:1020A90004F012529BE4906476F0A37412F09066E7
:1020B9007BE0906478F0A374FDF090610563A20160
:1020C90090647A63A2017F121235BF809812001EB4
:1020D9008F50E550B401159060007483F0E4A3F0CB
:1020E9007E607F007D02124A42021DDAE550D394D8
:1020F90001401C9060007483F0A37401F0E5502442
:10210900FEA3F07E607F007D03124A42021DDAE5DC
:102119000A64016003021DDA906576E004F0200B81
:10212900077E287F5F124259906356E0C3941E5080
:1021390004E02402F0906576E0C39405400DC203E3
:10214900E4906578F012529D021DDA7C667D8390D9
:10215900634AE0FAA3E0FB7F02124BD37E647F76E9
:10216900906477E02404FD124A42906356E0F50A30
:10217900021DDAE50A64016003021DDA906578E060
:1021890014604624FE604214700302226F24046026
:1021990003021DDAE4F50C200F139065787404F03E
:1021A900906576E05401F0750A01021DDA9080020B
:1021B9007410F0E4906578F090657604F0750A1271
:1021C90090668374FFF0021DDA906683E070030263
:1021D90022599064767480F09064787401F0E4A3D5
:1021E900F0A304F0A37430F0A3747BF0E4F5507409
:1021F9007D2550F582E43464F583747DF0747E2581
:1022090050F582E43464F583E4F0E55024079064E2
:1022190077F07C667D8390634AE0FAA3E0FB7F0256
:10222900124BD37E647F76E5502409FD124A429011
:102239006682E0601B12529CD203E4F50A9065762F
:10224900F090668704F0E490667AF0A3F0021DDA54
:10225900300F07E4906578F080069065787404F093
:10226900750A12021DDA9080027410F0750A039043
:102279006576E06401FFF09065787401F0EF7019FC
:10228900906352E06013FCA3E0FDA3E0FEA3E0FF2E
:102299009066831231C9021DDA90634EE0FCA3E017
:1022A900FDA3E0FEA3E0FF9066831231C9021DDAA7
:0222B90080FEA5
:0122BB002200
:100AD400906377E0B444047F0180027F00906376E2
:100AE400E0B447047E0180027E00EE5F604A9063BA
:100AF4003FE0906378F0906340E0906379F0906316
:100B040041E090637AF0906342E090637BF09063FD
:100B140043E090637CF0906344E090637DF09063E5
:100B2400777452F09062AE63A2019080A863A20130
:100B34007F061235BF021383906332E0C3940850DA
:100B44000302138C90633FE0FF906378E06F6003CF
:100B540002138C906340E0FF906379E06F600302BE
:100B6400138C906341E0FF90637AE06F600302139B
:100B74008C906342E0FF90637BE06F600302138C10
:100B8400906343E0FF90637CE06F600302138C90FA
:100B94006344E0FF90637DE06F600302138C906315
:100BA40077E06444701A9080A8E0B4FF139062AEBA
:100BB40063A2019080A863A2017F061235BF801052
:100BC4009062B2E09080ACF09062B3E09080ADF0BF
:100BD40090668EE060037401F090668F7464F09008
:100BE40063777452F0906376E0646D6003020D26BF
:100BF4007BFF7A28796A122D317BFF7A28798490D9
:100C0400633FE0F559A3E0F55AA3E0F55BA3E0F5F3
:100C14005CA3E0F55DA3E0F55E122D317559FF7517
:100C24005A28755BE1755CFF755D28755EED7BFF89
:100C34007A2879BA122D317BFF7A2879F6122D3170
:100C44007BFF7A29795C122D317BFF7A297989908F
:100C54006345E0F559A3E0F55AA3E0F55BA3E0F59D
:100C64005C122D317BFF7A2979B390634EE0F559FC
:100C7400A3E0F55AA3E0F55BA3E0F55C122D317B0C
:100C8400FF7A2979E1906352E0F559A3E0F55AA37C
:100C9400E0F55BA3E0F55C122D317BFF7A2A790F36
:100CA40090633BE0F559A3E0F55AA3E0F55BA3E0BC
:100CB400F55C122D317BFF7A2A7932906337E0F5A7
:100CC40059A3E0F55AA3E0F55BA3E0F55C122D31DE
:100CD4007BFF7A2A794F122D317BFF7A2A7978A209
:100CE4000FE433F559122D317BFF7A2A79A89066E7
:100CF40082E0F559122D317BFF7A2A79D390668EE2
:100D0400E0F559122D317BFF7A2B79069062B4E01D
:100D1400F559122D311236CD7BFF7A2B7938122DED
:100D24003122906376E0644C70737E2B7F3EFBFD32
:100D3400FC123F5E90637EE0F551A3E0F552E4F5CA
:100D440054E551906380F0A3E552F07E2B7F797CCB
:100D5400637D807B02123F5EE4F5538552828551A8
:100D640083E0FF74802553F582E43463F583EFF068
:100D74000552E552700205510553E553B410DC7E6B
:100D84002B7F7C7C637D807B10123F5E0554E55491
:100D9400C3941040AC7E2B7F7F124259229063761D
:100DA400E0646C7060F5557E2B7F81FBFDFC123F87
:100DB4005EE4F554E4906380F0A3E555F07E2B7F68
:100DC400797C637D807B02123F5EE4F553A855E68F
:100DD400FF74802553F582E43463F583EFF0055501
:100DE4000553E553B410E67E2B7F7C7C637D807BCA
:100DF40010123F5E0554E554C3940840B77E2B7F20
:100E04007F12425922906376E0644B7061F553740B
:100E1400682553F582E43463F583E0603274682511
:100E240053F582E43463F583E0F460237468255356
:100E3400F582E43463F583E0FF747E2553F582E4A0
:100E44003463F583E0B507100553E553B408C09047
:100E540061047432F00213839063767421F0300BD2
:100E6400030213837E2B7FBC1242590213839063C7
:100E740076E0B4521A200B077E2B7FC4124259909D
:100E840063767472F07E637F767D081249BB22908C
:100E94006376E064497045200B077E2B7FCF1242B6
:100EA4005990637EE0F551A3E0F552E4F553855281
:100EB40082855183E0FF74802553F582E43463F521
:100EC40083EFF00552E552700205510553E553B422
:100ED40080DC7E637F767D8A1249BB22906376E054
:100EE40064437046200B077E2B7FD71242599063D0
:100EF4007EE0F551A3E0F552E4F553855282855125
:100F040083E493FF74802553F582E43463F583EF1F
:100F1400F00552E552700205510553E553B480DBE8
:100F24007E637F767D8A1249BB22906376E0645AA1
:100F34007053200B077E2B7FE012425990637EE0B2
:100F4400F551A3E0F5527C637D807B80AF52AE51B6
:100F540012514AE4F553855282855183E493FF7418
:100F6400802553F582E43463F583EFF00552E552AE
:100F7400700205510553E553B480DB7E637F767DB3
:100F84008A1249BB22906376E06444600302101A1B
:100F940090637EE0FF64447003021383EFB4310C6A
:100FA400C20B7E2B7FEC12425902138390637EE0C6
:100FB400B4300CD20B7E2B7FF8124259021383906B
:100FC400637EE0B4320CD20C7E2C7F0512425902AF
:100FD400138390637EE0B4330CC20C7E2C7F131217
:100FE400425902138390637EE0B4340CD20D7E2CFC
:100FF4007F2212425902138390637EE0B4350CC2FF
:101004000D7E2C7F2F12425902138390637EE0FFE2
:10101400120021021383906104E07013200B077EF9
:101024002C7F3D1242599063767421F00213839011
:1010340061047432F0906376E0FFB45104C2AF806F
:10104400FEEF64577045200B077E2C7F4B124259EC
:1010540090637FE0906332F0E4F553906332E0FFF5
:10106400E553C39F400302138374802553F582E440
:101074003463F583E0FF90637EE0255324ADF5826D
:10108400E43461F583EFF0055380D0906376E06437
:1010940053600302113D200B077E2C7F56124259E8
:1010A40090633FE0FF9061B6E06F703C906340E076
:1010B400FF9061B7E06F7030906341E0FF9061B8DA
:1010C400E0B50724906342E0FF9061B9E0B50718EA
:1010D400906343E0FF9061BAE0B5070C906344E08D
:1010E400FF9061BBE06F60169063767421F0300B63
:1010F400030213837E2C7F65124259021383E4F5A5
:1011040053E4F50DAF53FE74AD2553F582E4346119
:10111400F583E0FD1251A40553E553C394FE40E169
:10112400C2AFE4907FF0F0A3F0907FFD74AAF0A327
:1011340074FFF0A37455F080FE906376E0644F7002
:101144005A90637EE0F551A3E0F552E552455170A3
:101154000A200B077E2C7F6E124259200B077E2C2F
:101164007F75124259E4F55374802553F582E434B3
:1011740063F583E0855282855183F00552E5527010
:101184000205510553E553B480DE90668DE024805A
:10119400F090668CE03400F0021383906376E06490
:1011A40045707490637EE0FEA3E0FF907FF0EEF064
:1011B400A3EFF0D39400EE94044038907FF0E0FE67
:1011C400A3E0FF90668CE0FCA3E0FD9FEC9E40232F
:1011D400E42FFFEE3401FED3ED9FEC9E5015C2AF19
:1011E400907FFD74AAF0A374FFF0A37455F0E4F5A6
:1011F400A780FE7E2C7F771242597BFF7A2C797F61
:10120400907FF0E0F559A3E0F55A90668CE0F55B29
:10121400A3E0F55C122D31906376E064656003020F
:10122400138C90637EE0FFA3E0907FF0CFF0A3EFF8
:10123400F0E4F551F552D3907FF1E09552907FF0B0
:10124400E095514020E4F50D2552FFE5513401FEAF
:10125400855282855183E0FD1251A40552E55270F6
:1012640002055180D17E2C7F8A124AC9EF4E60203C
:10127400120003906345EFF0120003906346EFF011
:10128400120003906347EFF0120003906348EFF0FD
:101294007E2C7F90124AC9EF4E60201200039063A7
:1012A4004EEFF012000390634FEFF01200039063CF
:1012B40050EFF0120003906351EFF07E2C7F9612F2
:1012C4004AC9EF4E6020120003906352EFF01200FF
:1012D40003906353EFF0120003906354EFF0120095
:1012E40003906355EFF07E2C7F9C124AC9EF4E6049
:1012F4002012000390633BEFF012000390633CEF75
:10130400F012000390633DEFF012000390633EEF90
:10131400F07E2C7FA2124AC9EF4E60201200039087
:101324006337EFF0120003906338EFF0120003907C
:101334006339EFF012000390633AEFF0E4F553E4FD
:10134400F50DE5532401FFE433FE74372553F5828C
:10135400E43463F583E0FD1251A40553E553C394CB
:101364004340DCC2AFE4907FF0F0A3F0907FFD74C3
:10137400AAF0A374FFF0A37455F0E4F5A780FE7EF1
:08138400637F767D081249BB6E
:01138C00223E
:10511200AE07EEC39430400BEED394395005EE2423
:10512200D0FF22EEC39461400BEED394665005EE9D
:1051320024A9FF22EEC39441400BEED394465005BE
:08514200EE24C9FF22AF062292
:10526A009062ADE004F070069062ACE004F09062E7
:0A527A00ACE0FEA3E0FF1252302268
:1000030012526A125112EFC454F0FEC00612526A21
:08001300125112D0E02FFF2270
:104F7200E4906CE9F012526A906CEAEFF0C394305C
:104F82004018E0FFD394395011906CE9E02405F504
:104F920082E43461F583EFF08011906CE9E024053E
:104FA200F582E43461F583E4F0800C906CE9E0046E
:104FB200F0E0D3940840BE75550075560075570051
:0C4FC200E4F5587B017A61790512389003
:014FCE0022C0
:044AC9008E568F571F
:104ACD009062ACE4F0A374FFF012526AEF606EF4E2
:104ADD00606B855782855683E493B507EC75580155
:104AED00E5572558F582E43556F583E49360259016
:104AFD0062ADE02558FF9062ACE03400FE125230FA
:104B0D00E5572558F582E43556F583E493B507044A
:104B1D00055880CCE5572558F582E43556F583E4E4
:104B2D009370A6E55824FFFFE434FFFE9062ADE0DC
:104B3D002FF09062ACE03EF07E007F0122E4FEFF9C
:014B4D002245
:104341007E2C7FA8124AC9EF4E70037F01227E2C7A
:104351007FAB124AC9EF4E600C12526AEF24D0248F
:10436100FF920F8002D20F7E2C7FB1124AC9EF4E0D
:10437100600C12526AEF24D0906682F08005E490BE
:104381006682F07E2C7FB7124AC9EF4E600C125242
:104391006AEF24D090668EF08005E490668EF07E00
:1043A1002C7FBD124AC9EF4E600C12526AEF24D025
:1043B10024FF92018002C2017E2C7FC3124AC9EF01
:1043C1004E600C12526AEF24D09062B4F08005E482
:1043D1009062B4F090633F63A20190667C63A20196
:1043E1007F061235BF30013B7E2C7FC9124AC9EFCF
:1043F1004E603012000390667CEFF012000390666D
:104401007DEFF012000390667EEFF01200039066DC
:104411007FEFF0120003906680EFF01200039066C8
:0644210081EFF07F002294
:10508500906577E0C3947C40027F0A906577E0FEE7
:1050950004F074B52EF582E43462F583EFF0BF0AAF
:1050A50027906577E0FF04F074B52FF582E434624C
:1050B500F583E4F0906577E0FF124B4E90657774C9
:0950C50008F09062B6E004F0224C
:10502B009080007480F090633763A201F583F58262
:10503B0063A2017F081235BF90633F63A20190808A
:10504B008863A2017F0A1235BF9080927407F0A388
:10505B0074D0F0A37406F0906349E0FF9080B1F038
:10506B009080E1EFF09080957455F0A3F090800064
:0A507B007401F090800974F0F02237
:104E4100908009E04410F09080A0E070609080A113
:104E51007482F09080A874FFF0A3F0A3F0A3F07F18
:104E6100039080AEEFF0A374CBF09080007402F059
:104E7100906CDD1231D500000000906CDDE0908077
:104E810040F0906CDEE0908041F0906CDFE090802B
:104E910042F0906CE0E0908043F0A3E4F0A3F0A333
:0D4EA100F0A3F0908018F0A3F0A3F0A3F0B0
:014EAE0022E1
:104FCF00908009E04440F09080D17482F07F03908C
:104FDF0080DEEFF0A374CCF09080027402F0906C3E
:104FEF00E11231D500000000906CE1E0908058F0A4
:104FFF00906CE2E0908059F0906CE3E090805AF072
:10500F00906CE4E090805BF0A3E4F0A3F0A3F0A336
:0B501F00F0908030F0A3F0A3F0A3F0AD
:01502A002263
:104D5500908009E04420F09080B8E0706C9080B9B4
:104D65007482F07F039080C6EFF07FCDA3EFF07FD4
:104D7500039080C4EFF0A374CDF09080C074FFF071
:104D8500A3F0A3F0A3F09080017402F0906CE512FB
:104D950031D500000000906CE5E090804CF0906CFF
:104DA500E6E090804DF0906CE7E090804EF0906CDE
:104DB500E8E090804FF0A3E4F0A3F0A3F0A3F09017
:094DC5008024F0A3F0A3F0A3F098
:014DCE0022C2
:104BD3008C518D52A907EAFDE975F018A424ACFFA6
:104BE300E5F034808F82F583EDF0EBFDE975F01885
:104BF300A4FFAEF024ACFBEE34808B82F583A3EDEF
:104C0300F08552828C83E0FDEF24A8FFEE3480FE12
:104C13008F82F583EDF08552828C83A3E08F828EA1
:104C230083A3F0855282855183A3A3E0FDE975F048
:104C330018A424A8FFE5F03480FE8F82F583A3A394
:104C4300EDF08552828C83A3A3A3E08F828E83A38E
:044C5300A3A3F02205
:0649BB008D56AB07AA06B1
:1049C100908000E030E5079065797401F022906CE9
:1049D100DDE0FCA3E0FDA3E0FEA3E0F55A8E598DD6
:1049E100588C57AE02AF038E838F8263A201E559C3
:1049F100540744C0F583855A8263A201AF5612362B
:104A010031E4FCFDFEE55A2556F55AEE3559F559C6
:104A1100ED3558F558EC3557F557908040E557F08E
:104A2100A3E558F0A3E559F0A3E55AF0908000748E
:104A310020F0AF5AAE59AD58AC57906CDD1231C968
:014A41002252
:064A42008D51AB07AA062E
:104A4800908002E030E5079065797403F022906C5D
:104A5800E1E0FCA3E0FDA3E0FEA3E0F5558E548D54
:104A6800538C52AE02AF038E838F8263A201E5544A
:104A7800540744D0F58385558263A201AF5112369D
:104A880031E4FCFDFEE5552551F555EE3554F55458
:104A9800ED3553F553EC3552F552908058E552F008
:104AA800A3E553F0A3E554F0A3E555F09080027414
:104AB80020F0AF55AE54AD53AC52906CE11231C9F1
:014AC80022CB
:0246BF008F5119
:1046C100908001E030E5099065797402F07F002265
:1046D100906CE5E0FCA3E0FDA3E0FEA3E0F5558EC0
:1046E100548D538C5290667C63A201E55454074467
:1046F100C8F58385558263A2017F06123647E555C9
:104701002406F555E43554F554E43553F553E435B1
:1047110052F55290657A63A201E554540744C8F5F5
:104721008385558263A201AF51123647E4FCFDFE39
:10473100E5552551F555EE3554F554ED3553F55301
:10474100EC3552F55290804CE552F0A3E553F0A3BD
:10475100E554F0A3E555F09080017420F0AF55AE1B
:0D47610054AD53AC52906CE51231C9AF510C
:01476E002228
:104065009081E0E0F5510551055105510551055186
:1040750005510551055105510551908010E0F55444
:10408500A3E0F555A3E0F556A3E0F5579081E1E0EF
:10409500F55105510551055105510551055105517B
:1040A500055105510551908014E0F558A3E0F559E7
:1040B500A3E0F55AA3E0F55BE55AB55608E55BB50F
:1040C50057037F0022E4F551E55A540744E0F58390
:1040D500855B8263A20190637663A2017F08123635
:1040E5007790637863A2019062AE63A2017F0612A6
:1040F50035BF906376E0F552A3E0F553E4F55190B2
:104105006376E0702AA3E024F8F551E55A54074494
:10411500E0F583855B8274082582F582E43583F5B5
:104125008363A20190637663A201AF51123677AE25
:1041350052E4FCFDE55B2553F55BE55A3EF55AED8A
:104145003559F559EC3558F558908014E558F0A3D4
:10415500E559F0A3E55AF0A3E55BF09080007440C3
:03416500F0AF5167
:014168002234
:103A34009081E6E0F55105510551055105510551B7
:103A440005510551055105510551908028E0F55463
:103A5400A3E0F555A3E0F556A3E0F5579081E7E020
:103A6400F5510551055105510551055105510551B2
:103A740005510551055190802CE0F558A3E0F55906
:103A8400A3E0F55AA3E0F55BE4F551E55AB5560A0F
:103A9400E55BB55705C208023BA0E55A540744F05C
:103AA400F583855B8263A20190637663A2017F083C
:103AB400123677906376E0F552A3E0F553E553456B
:103AC4005270099080027410F07F0022906683E0A7
:103AD400FFF46030906378E06F6003023B679066A8
:103AE40084E0FF906379E06F7079906685E0FF90E1
:103AF400637AE06F706D906686E0FF90637BE06FA1
:103B04006031805F906378E0906683F0906379E041
:103B1400906684F090637AE0906685F090637BE031
:103B2400906686F090637CE0FFA3E090634ACFF058
:103B3400A3EFF0906376E0702AA3E024F8F551E552
:103B44005A540744F0F583855B8274082582F58214
:103B5400E43583F58363A20190637663A201AF51D8
:103B6400123677AE52E4FCFDE55B2553F55BE55A6E
:103B74003EF55AED3559F559EC3558F558AF57AE71
:103B840056AD55AC54AB5BAA5AA959A858D31231B7
:103B9400A540099080027410F07F002290802CE5EB
:103BA40058F0A3E559F0A3E55AF0A3E55BF0908043
:063BB400027440F0AF5165
:013BBA0022E8
:103BBB009081E3E0F5510551055105510551055132
:103BCB000551055105510551055190801CE0F554E7
:103BDB00A3E0F555A3E0F556A3E0F5579081E4E09B
:103BEB00F55105510551055105510551055105512A
:103BFB00055105510551908020E0F558A3E0F5598A
:103C0B00A3E0F55AA3E0F55BE4F551E55AB5560A86
:103C1B00E55BB55705C209023D11E55A540744E867
:103C2B00F583855B8263A20190600463A2017F0E22
:103C3B0012368D906004E0F552A3E0F55390600CC2
:103C4B00E0FFF4604A90667CE0FEEF6E7079A3E0D3
:103C5B00FF90600DE06F706F90667EE0FF90600EDE
:103C6B00E06F706390667FE0FF90600FE06F7057BE
:103C7B00906680E0FF906010E06F704B906681E083
:103C8B00FF906011E06F703FE4906013F08008903C
:103C9B00601374FFF0D2D9906004E0702AA3E02483
:103CAB00F2F551E55A540744E8F583855B82740EAF
:103CBB002582F582E43583F58363A201906004636A
:103CCB00A201AF5112368DAE52E4FCFDE55B2553DC
:103CDB00F55BE55A3EF55AED3559F559EC3558F586
:103CEB0058AF57AE56AD55AC54AB5BAA5AA959A8B1
:103CFB0058D31231A55006E55345527009908001F7
:103D0B007410F07F0022908020E558F0A3E559F065
:103D1B00A3E55AF0A3E55BF09080017440F0AF513E
:013D2B002275
:044259008E568F5797
:10425D00908000E030E5079065797401F022906C54
:10426D00DDE0FCA3E0FDA3E0FEA3E0F55D8E5C8D3B
:10427D005B8C5AE55DFFE55C5407FEE42FF559EEC6
:10428D0034C0F558855982F5837423F00559E559E5
:10429D00700205585358C7F582855883740AF00586
:1042AD0059E559700205585358C790633F63A201F1
:1042BD0085588385598263A2017F061236317406B3
:1042CD002559F559E43558F5588556838557826338
:1042DD00A20185588385598263A201123615E4FC2B
:1042ED00FDFE906CDDE0F8A3E0F9A3E0FAA3E02F6A
:1042FD00FFEE3AFEED39FDEC38FCEF2408FFE43E0D
:10430D00FEE43DFDE43CFC906CDD1231C9906CDDAA
:10431D00E0908040F0906CDEE0908041F0906CDF9A
:10432D00E0908042F0906CE0E0908043F09080004F
:03433D007420F0F9
:01434000225A
:0A3F5E008E568F578C588D598B5AE0
:103F6800908000E030E5079065797401F022906C4C
:103F7800DDE0FCA3E0FDA3E0FEA3E0F5608E5F8D2D
:103F88005E8C5DE560FFE55F5407FEE42FF55CEEAF
:103F980034C0F55B855C82F5837423F0055CE55CD1
:103FA8007002055B535BC7F582855B83740AF00575
:103FB8005CE55C7002055B535BC790633F63A201DD
:103FC800855B83855C8263A2017F061236317406A5
:103FD800255CF55CE4355BF55B8556838557826324
:103FE800A201855B83855C8263A2011236158F610D
:103FF800EF255CF55CE4355BF55BE55A60178558A1
:104008008385598263A201855B83855C8263A201F3
:10401800AF5A123631E5612408255AF55AFFE4FCF7
:10402800FDFEE5602FF560EE355FF55FED355EF579
:104038005EEC355DF55D908040E55DF0A3E55EF0F2
:10404800A3E55FF0A3E560F09080007420F0AF6016
:0C405800AE5FAD5EAC5D906CDD1231C956
:014064002239
:0645E4008E538F548D552B
:1045EA00908000E030E5079065797401F022906CC4
:1045FA00DDE0FCA3E0FDA3E0FEA3E0F55B8E5A8DAF
:10460A00598C58E55BFFE55A5407FEE42FF557EE3F
:10461A0034C0F556855782F5837423F00557E5575C
:10462A00700205565356C7F582855683EBF0055737
:10463A00E557700205565356C790633F63A201853A
:10464A00568385578263A2017F0612363174062586
:10465A0057F557E43556F55685538385548263A238
:10466A000185568385578263A201AF55123631748C
:10467A00082555F555FFE4FCFDFEE55B2FF55BEEDD
:10468A00355AF55AED3559F559EC3558F5589080A3
:10469A0040E558F0A3E559F0A3E55AF0A3E55BF02D
:1046AA009080007420F0AF5BAE5AAD59AC58906C54
:0446BA00DD1231C913
:0146BE0022D9
:024B4E008F6A6C
:104B5000908000E030E5079065797401F022906C58
:104B6000DDE0FCA3E0FDA3E0FEA3E0F56E8E6D8D1D
:104B70006C8C6BE56EFFE56D5407FEE42FFFEE34A1
:104B8000C09062B563A201F5838F8263A201AF6A10
:104B9000123631E4FCFDFEE56E256AF56EEE356DEC
:104BA000F56DED356CF56CEC356BF56B908040E593
:104BB0006BF0A3E56CF0A3E56DF0A3E56EF09080DB
:104BC000007420F0AF6EAE6DAD6CAC6B906CDD120E
:024BD00031C9E9
:014BD20022C0
:064427008E558F56AB0517
:10442D00908000E030E5079065797401F022906C82
:10443D00DDE0FCA3E0FDA3E0FEA3E0F55C8E5B8D6B
:10444D005A8C59E55CFFE55B5407FEE42FF558EEF9
:10445D0034C0F557855882F5837423F00558E55817
:10446D00700205575357C7F582855783EBF00558F2
:10447D00E5587002055790633F63A2018557838508
:10448D00588263A2017F0612363174062558F558FD
:10449D00E43557F5575357C7E555855882855783EA
:1044AD00F00558E558700205575357C7F5828557E3
:1044BD0083E556F00558E558700205575357C7E583
:1044CD005C240AF55CE4355BF55BE4355AF55AE49A
:1044DD003559F559908040E559F0A3E55AF0A3E51B
:1044ED005BF0A3E55CF09080007420F0AF5CAE5BF8
:0A44FD00AD5AAC59906CDD1231C9C4
:014507002291
:104EAF00908009E04480F09080E97441F07F099090
:104EBF0080F6EFF0A37464F09080037402F090809A
:104ECF0003E020E1F9906BD91231D500000000907A
:104EDF006BD9E0908064F0906BDAE0908065F09091
:104EEF006BDBE0908066F0906BDCE0908067F0A366
:104EFF00E4F0A3F0A3F0A3F090803CF0A3F0A3F0B4
:024F0F00A3F00D
:014F1100227D
:104508009081E9E0F55305530553055305530553C9
:1045180005530553055305530553908034E0F5546E
:10452800A3E0F555A3E0F556A3E0F5579081EAE03E
:10453800F5530553055305530553055305530553C3
:10454800055305530553908038E0F558A3E0F55915
:10455800A3E0F55AA3E0F55BE55AB55608E55BB567
:1045680057037F0022AF5BAE5AAD59AC58AB57AA80
:1045780056A955A854D31231A5400AAF5BAE57EEE1
:104588009FF553800AAF5BEFF404AE572EF553E561
:104598005A540744E0F583855B8263A201906BDD82
:1045A80063A201AF531236A5E4FCFDFEE55B25537B
:1045B800F55BEE355AF55AED3559F559EC3558F5A0
:1045C80058908038E558F0A3E559F0A3E55AF0A3D0
:0B45D800E55BF09080037440F0AF53EF
:0145E30022B5
:024169008F5372
:10416B009080E8E0640660037FFF22906BD9E0FC4F
:10417B00A3E0FDA3E0FEA3E0F5578E568D558C54BE
:10418B00E4FFFEFDFCAB57AA56A955A854C3123148
:10419B00A570609081F9E0F554906BD9E0FCA3E039
:1041AB00FDA3E0FEA3E0FFE4FAF9F8EF2401FFEA38
:1041BB003EFEE93DFDE83CFC906BD91231C9906B9A
:1041CB00D9E0FCA3E0FDA3E0FEA3E0FFE4F8EF24BD
:1041DB0001FFEA3EFEE93DFDE83CFC906BD9123154
:1041EB00C9908064E0F554A3E0F555A3E0F556A320
:1041FB00E0F557906BDD63A201E556540744D8F503
:10420B008385578263A201AF5312365FE4FCFDFE38
:10421B00E5572553F557EE3556F556ED3555F5550E
:10422B00EC3554F554908064E554F0A3E555F0A3B8
:10423B00E556F0A3E557F09080037420F0AF57AE2E
:0D424B0056AD55AC54906BD91231C97F00AF
:014258002243
:10523000A2AF9210C2AF438E2075D2028F828E83AE
:0C524000E0FFE4F5D2538EDFA21092AF25
:01524C00223F
:1051A400E5D220E0FBA2AF9210C2AF43D2028F82BD
:1051B4008E83EDF075D25063D250A21092AFE5D237
:0351C40020E0FBED
:0151C70022C5
:104CD700E4FDED2401FFE433FE12523074372DF565
:104CE70082E43463F583EFF00DBD3FE6E4FDED2488
:104CF7007FFFE433FE125230742D2DF582E43461C8
:104D0700F583EFF0742D2DF582E43461F583E070BF
:104D17001B742D2DF582E43461F5837420F0742E15
:104D27002DF582E43461F583E4F080040DBD80BE87
:104D3700E49061ACF0FDEDFF7E0012523074AD2DB2
:0D4D4700F582E43461F583EFF00DBDFEE967
:014D5400223C
:02514A008B5682
:10514C00A2AF9210C2AF85A25753A2FE8E838F825C
:10515C0005A28C838D8274091236BBE55653A2FED0
:10516C0043A2201236BD53A2DF8557A2A21092AFE4
:01517C00FF33
:01517D00220F
:10524D00A2AF9210C2AF8C838D82EF1236BB43A2F8
:0C525D00201236BD53A2DFA21092AFFF5A
:015269002222
:0251C8008F5105
:1051CA00A2AF9210C2AFE4F5838D8274061236BB89
:1051DA00E55143A2201236BD53A2DFA21092AF7F3F
:0151EA0001C3
:0151EB0022A1
:0251EC008F51E1
:1051EE00A2AF9210C2AFE4F5838D82740A1236BB61
:1051FE00E55143A2201236BD53A2DFA21092AF7F1B
:01520E00019E
:01520F00227C
:1034E400A907E7FFA805EF93C3966008403B74FC67
:1034F4002FFF80F00F08EF93C3966008402B74FBF6
:103504002FFF80E00F08EF93C3966008401B74FA06
:103514002FFF80D00F08EF93D3966008400B74F907
:103524002FFF80C01F1F1F1F1FEF54FEF80303F758
:10353400E893FC08E893FD08E893FE08E893FF226B
:1035440009E993C39D6008402974FB29F980F109B6
:10355400E993C39E6008401A74FA29F980E209E9E4
:1035640093D39F6008400B74F929F980D319191972
:103574001919E9C313C313FF22740093F8ECC39819
:103584004024701F740193F8EDC3984019701474AB
:0E3594000293F8EEC398400E7009740393F88A
:1035A200EFC39840037F00227F0122EDF8E6F00886
:1035B200A3DFFA22EDF8E0F608A3DFFA22E0A36324
:1035C200A201F0A363A201DFF475A2002263A201AB
:1035D200F0A363A20122E0A363A201F0A363A2010C
:1035E200E0A363A201F0A363A201E463A201F0A33A
:1035F20063A201DFE175A20022E0A363A2016DFED6
:10360200936CFDEE058393FC158363A201DFEA75DB
:10361200A200227F00E493A363A201F00F600CA337
:10362200E583C2E3F58363A20180EA75A20022E08A
:10363200A363A201F0A3E583C2E3F58363A201DFE2
:10364200EE75A20022E0A363A201F0A3E583C2E427
:10365200D2E3F58363A201DFEC75A20022E0A3634B
:10366200A201F0A3E58344F8C2E5F58363A201DF7A
:10367200EC75A20022E583C2E3F583E0A363A20115
:10368200F0A363A201DFEE75A20022E583C2E4D2B9
:0A369200E3F583E0A363A201F0A3B7
:10369C0063A201DFEC75A20022E58344F8F583E018
:1036AC00A363A201F0A363A201DFEE75A20022F9CD
:1036BC0022C002C004C00612FFF0D006D004D00213
:0136CC0022DB
:1022BC003E2A2C312CCFE0F0E0ECE5F2F0FB20F8DC
:1022CC00E8EDFB2043414E0A003E4C2C6B30312C88
:1022DC0025732C43EAEEF0EEF1F2FC20EDE020F851
:1022EC00E8EDE52043414E2C30202D20353030EAEE
:1022FC00E1283530EC292C31202D203530EAE1282D
:10230C00353030EC290A0030202D20353030EAE110
:10231C00283530EC290031202D203530EAE12835E4
:10232C003030EC29003E2A2C312CCFE0F0E0ECE5EB
:10233C00F2F0FB20EFF0EEF2EEEAEEEBE020D1DD76
:10234C00D22D34D2CC28CCE5F0EAF3F0E8E93233E4
:10235C0030290A003E422C4930322C2562752CD291
:10236C00E8EF20EFF0EEF2EEEAEEEBE020CCE5F059
:10237C00EAF3F0E8E90A003E532C4930332C25737C
:10238C002CCFE0F0EEEBFC20E4EEF1F2F3EFE00A00
:10239C00003E4C2C4930312C256C752CD1EAEEF0DA
:1023AC00EEF1F2FC20EEE1ECE5EDE02C31323030D8
:1023BC002C323430302C343830302C393630302C00
:1023CC0031393230300A003E422C4930352C2562EE
:1023DC00752CCAEEEDF2F0EEEBFC20EFEE20EDE505
:1023EC00F7E5F2EDEEF1F2E80A003E532C493132FA
:1023FC002C2562752CC0E4F0E5F120E1EBEEEAE06F
:10240C0020D2C8D220EDE020F8E8EDE50A003E53DA
:10241C002C4931332C256C752CCFE0F3E7E020EC04
:10242C00E5E6E4F320F6E8EAEBE0ECE820EEEFF08A
:10243C00EEF1E028F1E5EA290A003E532C4931344B
:10244C002C256C752CD6E8EAEB20EFE5F0E5E4E002
:10245C00F7E820D2C8D228F1E5EA290A003E532C2D
:10246C004931352C256C752CD6E8EAEB20EFE5F0DC
:10247C00E5E4E0F7E820D2C8C828ECE8ED290A002A
:10248C003E532C6D2562752C25732CCFF0E8E1EEB4
:10249C00F0202562752028C0E4F0E5F120E820EF5B
:1024AC00E0F0E0ECE5F2F0FB290A003C21003C6B8B
:1024BC0030313D003C4930333D003C4930313D002A
:1024CC003C4931323D003C4931333D003C493134CB
:1024DC003D003C4931353D003C4930323D003C49E2
:1024EC0030353D002043616E457247495400200A47
:1024FC00002043616E457272434821000A000AD6DF
:10250C00E8EAEB20EFF0EEF8E5EB0A000AC7E0EFA3
:10251C00F0EEF13A00496E69745443500A004C696C
:10252C007374656E5443500A00534F434B5F5443CE
:10253C00505F45535441424C49534845440A000AA4
:10254C002D3E20000A3C2D2000CFF0E8E5EC3A00AF
:10255C00CEF8E8E1EAE020CAD1210A00CED8C8C101
:10256C00CAC020C0E4F0E5F1E02100CED8C8C1CA51
:10257C00C020EEF2EAF0FBF2E8FF20EAE0EDE0EB3F
:10258C00E02100204F4B212000CED8C8C1CAC0206A
:10259C00E7E0EFF0EEF1E0000A3D0028253033646F
:1025AC002920256C64202020202020202020202081
:1025BC00200000C1814001C0804101C0804100C1A8
:1025CC00814001C0804100C1814000C1814001C0F7
:1025DC00804101C0804100C1814000C1814001C0E7
:1025EC00804100C1814001C0804101C0804100C1D7
:1025FC00814001C0804100C1814000C1814001C0C7
:10260C00804100C1814001C0804101C0804100C1B6
:10261C00814000C1814001C0804101C0804100C1A6
:10262C00814001C0804100C1814000C1814001C096
:10263C00804101C0804100C1814000C1814001C086
:10264C00804100C1814001C0804101C0804100C176
:10265C00814000C1814001C0804101C0804100C166
:10266C00814001C0804100C1814000C1814001C056
:10267C00804100C1814001C0804101C0804100C146
:10268C00814001C0804100C1814000C1814001C036
:10269C00804101C0804100C1814000C1814001C026
:1026AC00804100C1814001C0804101C0804100C116
:1026BC00814000C0C101C30302C2C60607C705C5DD
:1026CC00C404CC0C0DCD0FCFCE0E0ACACB0BC9094E
:1026DC0008C8D81819D91BDBDA1A1EDEDF1FDD1D5E
:1026EC001CDC14D4D515D71716D6D21213D311D18E
:1026FC00D010F03031F133F3F23236F6F737F535DE
:10270C0034F43CFCFD3DFF3F3EFEFA3A3BFB39F90D
:10271C00F83828E8E929EB2B2AEAEE2E2FEF2DEDDD
:10272C00EC2CE42425E527E7E62622E2E323E1214D
:10273C0020E0A06061A163A3A26266A6A767A5655D
:10274C0064A46CACAD6DAF6F6EAEAA6A6BAB69A9CD
:10275C00A86878B8B979BB7B7ABABE7E7FBF7DBDDD
:10276C00BC7CB47475B577B7B67672B2B373B1710D
:10277C0070B05090915193535292965657975595DD
:10278C0094549C5C5D9D5F9F9E5E5A9A9B5B99598D
:10279C005898884849894B8B8A4A4E8E8F4F8D4D5D
:1027AC004C8C4484854587474686824243834181CD
:1027BC0080403C6D303D000000003C6D313D000020
:1027CC0000003C6D323D000000003C6D333D0000CC
:1027DC0000003C6D343D000000003C6D353D0000B8
:1027EC0000003C6D363D000000003C6D373D0000A4
:1027FC0000003C6D383D000000003C6D393D000090
:10280C0000003C6D31303D0000003C6D31313D002D
:10281C0000003C6D31323D0000003C6D31333D0019
:10282C0000003C6D31343D0000003C6D31353D0005
:02283C0000009A
:0100210022BC
:03002300024DCFBC
:0B4DCF00C0E0C083C082C0D075D018C7
:104DDA00309827E5E92464F5EB30D707E5F904F5BF
:104DEA00FB800385F9FBD29174B52539F582E43449
:104DFA006AF583E599F00539C298309931E53EC3E1
:104E0A009538501BAF3E053E74B52FF582E4346BDE
:104E1A00F583E0FF521FA2D0B3929B8F99800DE5D4
:0E4E2A003EC395384006053ED296C290C2990E
:094E3800D0D0D082D083D0E0324A
:1036CD007BFF7A2279BC122D31906892E0701475CF
:1036DD0059FF755A23755B137BFF7A2279D5122D0D
:1036ED003180127559FF755A23755B227BFF7A2243
:1036FD0079D5122D317BFF7A237931122D317BFF54
:10370D007A237960A21DE433F559122D31755901D3
:10371D00755A6A755B6A7BFF7A237983122D319016
:10372D006BD7E0FEA3E0FFC3E49FFFE49EFEAB0773
:10373D00FA3395E0F9F87F007E8C7D0A7C0012311A
:10374D00058F5C8E5B8D5A8C597BFF7A23799D1288
:10375D002D317BFF7A2379D3A219E433F559122D3C
:10376D00317BFF7A2379F6906893E0F559122D316C
:10377D00E47B64FAF9F89068DAE0FCA3E0FDA3E0DD
:10378D00FEA3E0FF1231058F5C8E5B8D5A8C597B49
:10379D00FF7A24791A122D31906896E0FEA3E0FF8E
:1037AD00E4FCFD7B64FAF9F81231058F5C8E5B8DBC
:1037BD005A8C597BFF7A247946122D31906890E00E
:1037CD00FEA3E0FFE4FCFD7B3CFAF9F81231058F16
:1037DD005C8E5B8D5A8C597BFF7A247969122D3161
:1037ED00E4906CE9F0906CE9E0FFC3648094904044
:1037FD000302388F906A197420F0E4A3F0EF33952B
:10380D00E0FEEF7803C333CE33CED8F924BEF58274
:10381D0074273EAF82FE124AC9EF4E6041E4906CB0
:10382D00EBF012526A906CEAEFF0643C601BE0FF23
:10383D00A3E0FE04F0EEFD3395E0FC74192DF58246
:10384D00746A3CF583EFF080D9906CEBE0FF339513
:10385D00E0FE74192FF582746A3EF583E4F0906CE6
:10386D00E9E0F559755A01755B6A755C1904F55DEA
:10387D007BFF7A24798C122D31906CE9E004F002F3
:02388D0037F210
:01388F002216
:0650CE00AC05AB07AA06C9
:1050D400906A1874FFF0906A69F0AF041CEF602DB9
:1050E4000BEBAE0270010A14F5828E83E0FF906A26
:1050F40018E06FFF9025BE93FE906A69E06E906A97
:0D51040018F0EF9026BE93906A69F080CD00
:01511100227B
:044C5700A907AE03F8
:104C5B00E4906CE9F0906CE9E0FFC39440501B8545
:104C6B004582854483A3E5822FF582E43583F58362
:104C7B00E4F0906CE9E004F080DB854582854483A9
:104C8B007406F0A3E9F0854582854483A3A37408D9
:104C9B00F0EED39401400E854582854483A3A3A3F4
:104CAB007416F0800C854582854483A3A3A37414EA
:104CBB00F0E5452404F582E43544F583EDF0E54554
:0B4CCB00241CF582E43544F583EEF074
:014CD60022BB
:100026007E247FB7124AC9EF4E70037F0122E49007
:100036006892F07E247FBA124AC9EF4E601B1252B4
:100046006A8F51E551B43106906892740AF0E55111
:10005600B432069068927464F07E247FC0124AC956
:10006600EF4E603512526A906A6AEFF012526A9049
:100076006A6BEFF012526A906A6CEFF012526A9055
:100086006A6DEFF012526A906A6EEFF012526A9041
:100096006A6FEFF0E4A3F08013906A6A7431F0A3FC
:1000A600F0A3F0A3F0A3F0A3F0E4A3F07E247FC6B0
:1000B600124AC9EF4E6023124F72A804A905AA0678
:1000C600AB077F007E8C7D0A7C00123105123197CA
:1000D600906BD7EEF0A3EFF0800A906BD774FFF029
:1000E600A374B8F07E247FCC124AC9EF4E600A1280
:1000F6004F72906893EFF08005E4906893F07E2449
:100106007FD2124AC9EF4E6014124F72E47B64FA32
:10011600F9F812307A9068DA1231C9800A9068DAF2
:100126001231D500000000E4FFFEFDFC9068DAE025
:10013600F8A3E0F9A3E0FAA3E0FBC31231A5700A25
:100146009068DA1231D50000000A7E247FD8124A60
:10015600C9EF4E6016124F72E47B64FAF9F812305A
:100166007A906896EEF0A3EFF08007E4906896F038
:10017600A3F0906896E07002A3E0700A9068967407
:100186000BF0A374B8F07E247FDE124AC9EF4E60EE
:1001960016124F72E47B3CFAF9F812307A906890A6
:1001A600EEF0A3EFF08007E4906890F0A3F090687B
:1001B60090E07002A3E07008906890F0A3743CF0A1
:1001C6007E247FE4124AC9EF4E600D124F72EC4D49
:1001D6004E4F24FF921D8002C21D7E247FEA124AE2
:1001E600C9EF4E600C12526AEF24D024FF92198098
:1001F60002C219E4F544F545301D5F854582854404
:1002060083A374FEF0854582854483A3A37403F01B
:10021600854582854483A3A3A37408F0E54524019C
:10022600FFE43544FE7D031250CE906A18E0FFE5E8
:10023600452404F582E43544F583EFF0906A69E0DD
:10024600FFE5452405F582E43544F583EFF0854561
:10025600828544837405F00202F4854582854483D1
:10026600A374FEF0854582854483A3A37403F085B9
:100276004582854483A3A3A37408F0E5452404F5C9
:1002860082E43544F5837455F0E5452405F582E4AA
:100296003544F58374AAF0E5452406F582E4354431
:1002A600F5837433F0E5452407F582E43544F58398
:1002B60074CCF0E5452401FFE43544FE7D07125079
:1002C600CE906A18E0FFE5452408F582E43544F54A
:1002D60083EFF0906A69E0FFE5452409F582E4358D
:1002E60044F583EFF08545828544837409F07420D4
:1002F6002545F545E43544F544854582F583E4F026
:10030600906A1704F0E4F551AF51EF3395E0FEEF34
:100316007803C333CE33CED8F924BEF58274273E94
:10032600AF82FE124AC9EF4E7003020A1F124F72C5
:10033600906AB4EFF07003020A2D906AB4E0B4FF3D
:1003460002E4F0201D030204FD906AB4E0854582B4
:10035600854483A3F0854582854483A3A37401F075
:10036600854582854483A3A3A3F0906A6AE0FFE5EE
:10037600452404F582E43544F583EFF0906A6BE09A
:10038600FFE5452405F582E43544F583EFF0906AF0
:100396006CE0FFE5452406F582E43544F583EFF08D
:1003A600906A6DE0FFE5452407F582E43544F58360
:1003B600EFF0906A6EE0FFE5452408F582E43544E7
:1003C600F583EFF0906A6FE0FFE5452409F582E4D6
:1003D6003544F583EFF0E5452401FFE43544FE7D21
:1003E600091250CE906A18E0FFE545240AF582E42A
:1003F6003544F583EFF0906A69E0FFE545240BF597
:1004060082E43544F583EFF0906AB4E0FFE54524D5
:1004160010F582E43544F583EFF0E5452411F582C5
:10042600E43544F5837401F0E5452412F582E4359C
:1004360044F5837401F0906A6AE024D0FFE5452410
:1004460013F582E43544F583EFF0906A6BE024D02F
:10045600FFE5452414F582E43544F583EFF0906A10
:100466006CE024D0FFE5452415F582E43544F58398
:10047600EFF0906A6DE024D0FFE5452416F582E49E
:100486003544F583EFF0906A6EE024D0FFE545240D
:1004960017F582E43544F583EFF0906A6FE024D0D7
:1004A600FFE5452418F582E43544F583EFF0E5458C
:1004B6002410FFE43544FE1250CE906A18E0FFE5A2
:1004C600452419F582E43544F583EFF0906A69E036
:1004D600FFE545241AF582E43544F583EFF08545BA
:1004E60082854483740BF0E582241EF582E435830D
:1004F600F583E4F00205B7906AB4E0854582854449
:1005060083A3F0854582854483A3A37401F0906A92
:100516006AE0854582854483A3A3A3F0906A6BE0D5
:10052600FFE5452404F582E43544F583EFF0906A4F
:100536006CE0FFE5452405F582E43544F583EFF0EC
:10054600906A6DE0FFE5452406F582E43544F583BF
:10055600EFF0906A6EE0FFE5452407F582E4354446
:10056600F583EFF0906A6FE0FFE5452408F582E435
:100576003544F583EFF0E5452401FFE43544FE7D7F
:10058600081250CE906A18E0FFE5452409F582E48A
:100596003544F583EFF0906A69E0FFE545240AF5F6
:1005A60082E43544F583EFF0854582854483740AF9
:1005B600F0E545241CF582E43544F583E4F0742027
:1005C6002545F545E43544F544906A17E004F08581
:1005D6004582854483E4F012526AEF12320606D24F
:1005E6000006D2210633230A0D2A09C22F06523BE2
:1005F60006D23C09C23E07F7430806450797460759
:10060600D64907C74C075B50076A5109D952078874
:100616005308865407A655093E61096A620996631E
:1006260008466509147308CD74000005DD12526A88
:1006360075F008EFA42436F582E5F03426AF82FE85
:10064600124AC9EF4E6090124F72808BE545240125
:10065600FFE43544FE7D041250CE906A18E0FFE5B3
:10066600452405F582E43544F583EFF0906A69E0A8
:10067600FFE5452406F582E43544F583EFF0E545CC
:100686002401FFE43544FE7D061250CE906A18E040
:10069600FFE5452407F582E43544F583EFF0906ADB
:1006A60069E0FFE5452408F582E43544F583EFF07B
:1006B60074202545F545E43544F544906A17E00471
:1006C600F0854582854483E4F00205DD8545828513
:1006D6004483E06075E5452401FFE43544FE7D046E
:1006E6001250CE906A18E0FFE5452405F582E43500
:1006F60044F583EFF0906A69E0FFE5452406F5824C
:10070600E43544F583EFF0E5452401FFE43544FE86
:100716007D061250CE906A18E0FFE5452407F58263
:10072600E43544F583EFF0906A69E0FFE545240877
:10073600F582E43544F583EFF074202545F545E46C
:100746003544F544906A17E004F085458285448374
:10075600E4F0020A1F906AB4E0FF7B0FE4FD124C3E
:10076600570205DD906AB4E0FF7B0F7D04124C57FB
:10077600E545241EF582E43544F583E04410F00295
:1007860005DD906AB4E0FF7B0F7D08124C57020529
:10079600DD906AB4E0FF7B017D40124C570205DD17
:1007A600301D0F906AB4E0FF7B077D11124C570293
:1007B60005DD906AB4E0FF7B0E7D10124C570205F2
:1007C600DD906AB4E0FF7B0E7D14124C570205DD06
:1007D600301D0F906AB4E0FF7B077D21124C570253
:1007E60005DD906AB4E0FF7B0E7D20124C570205B2
:1007F600DD906AB4E0FF7B0F7D30124C570205DDB9
:10080600906AB4E0FF7B017D0F124C5785458285C7
:100816004483A3A37405F0854582854483A3A3A3DB
:10082600E4F0E5452404F582E43544F583E4F0E597
:1008360045241CF582E43544F583740FF00205DD8A
:10084600906AB4E0FF7B017D0F124C578545828587
:100856004483A3A37405F0854582854483A3A3A39B
:10086600E4F0E5452404F582E43544F583E4F0E557
:1008760045241CF582E43544F5837405F00205DD54
:10088600906AB4E0FF7B017D0F124C578545828547
:100896004483A3A37405F0854582854483A3A3A35B
:1008A600E4F012526AEF24D0FFE5452404F582E411
:1008B6003544F583EFF0E545241CF582E43544F52F
:1008C60083740FF00205DD906AB4E0FF7B017D0FB3
:1008D600124C57854582854483A3A37405F085454C
:1008E60082854483A3A3A3E4F012526AEF24D0FFC7
:1008F600E5452404F582E43544F583EFF0E5452427
:100906001CF582E43544F5837405F00205DD854562
:1009160082854483A3A3A37411F0E5452404F582DC
:10092600E43544F583E0F0E545241CF582E43544DE
:10093600F5837401F00205DD854582854483A3A312
:10094600A37411F0E5452404F582E43544F583E00B
:100956004401F0E545241CF582E43544F583740131
:10096600F00205DD854582854483A3A3A37411F0B7
:10097600E5452404F582E43544F583E04402F0E5D8
:1009860045241CF582E43544F5837401F00205DD47
:10099600854582854483A3A3A37411F0E545240409
:1009A600F582E43544F583E04403F0E545241CF57F
:1009B60082E43544F5837401F00205DD12526AEFD4
:1009C60024D0FFE545241DF582E43544F583EFF098
:1009D6000205DDE545241EF582E43544F583E0FF96
:1009E60030E412E545241EF582E43544F583EF44F0
:1009F60040F00205DDE545241EF582E43544F58325
:100A0600E04401F00205DDE545241EF582E43544A7
:100A1600F583E04402F00205DD0551C3E55164802B
:100A26009490500302030EE4F544F545FFF5518515
:100A36004582854483E07003020ACDA3A3E06408DF
:100A4600703EE545241FF582E43544F583E551F013
:100A5600E545241CF582E43544F583E0FEB4010245
:100A66000551EEB40F0674042551F551EEB40E0689
:100A760074032551F551EEB4070674032551F5515B
:100A8600854582854483A3A3E06405702CE545244F
:100A96001FF582E43544F583EFF0E545241CF58225
:100AA600E43544F583E0FEB401010FEEB40F04749F
:100AB600042FFFEEB405020F0F74202545F545E41B
:0D0AC6003544F544020A35E4F544F545FFDA
:010AD3002200
:10517E00C2A9438902758C48758A4875D90475DBB6
:10518E004875DC4875DD4875DE48E4F5E9F5F9C289
:06519E00D9D28CD2DE2202
:10480D0043AB01C2E8C2EAE4FFEFC454F0F5B1C313
:10481D00EF64809488500575B3D08003E4F5B3EF51
:10482D007026F5B275BC01F5BDF5BEF5BF75C4FFBB
:10483D00F5C5F5C6F5C7F5A3F5A3F5A3F5A3F5A342
:10484D00F5A3F5A3F5A38027E4F5B275BCC8F5BDB6
:10485D00F5BE75BF7875C4FFF5C5F5C675C778F596
:10486D00A3F5A3F5A3F5A3F5A3F5A3F5A3F5A30F61
:10487D00BF0E96906892E0FF25E0F5B475B50C7506
:10488D00B66C75A11275AB0275C13E75C3FF75C2CD
:01489D000317
:01489E0022F7
:104F120075B180E4F5B3F5B28527BCE5285403FFEB
:104F220033333354F8FFE52854E04FFFE529C41327
:104F320054074FF5BDE52933333354F8FFE52AC44E
:104F42001354074FF5BEE52A33333354F8F5BF85C2
:104F52002CA3852DA3852EA3852FA38530A3853170
:104F6200A38532A38533A3E52B540F2450F5B32236
:103E5100E59B541F6020200B1A7E247FF0124259EB
:103E6100E59B541FFF7E007D031244277E247FFAC9
:103E7100124259E4F59BE5BA30E008E4F5B375B1B7
:103E810080F5B2E5CFF47003023F5B755401E4F5B0
:103E910053E5CFF455547003023F49E553C454F040
:103EA100F5B1E5B2547F6420706FE5B3540FF52B83
:103EB10085BC27E5BD541FFF131313541FFFE5BD38
:103EC10054E044184FF528E5BDC43354E0FFE5BE86
:103ED100131313541F4FF529E5BEC43354E0FFE516
:103EE100BF131313541F4FF52A85A32C85A32D85CA
:103EF100A32E85A32F85A33085A33185A33285A366
:103F010033E4F5B2E527547EB5270575B350800338
:103F110075B3D0E52B2405FF22E5B2549F60232021
:103F21000B207E247FFD124259AFB27E007D031229
:103F31004427AFB37E007D031244277E257F0812FC
:103F41004259E4F5B275B3D0E55425E0F554055373
:0C3F5100E553C394085003023E927F0029
:013F5D002241
:10476F00C21AE4F539F50BD296F538F53EF525FF6B
:10477F0074742FF582E4346AF583E4F074982FF59E
:10478F0082E43468F583E4F00FBF40E4E49069E31A
:10479F00F0A3F0F53FF54F12002612480DC2ADE41D
:1047AF00F5C9D2CDD2CCC2C9C2CAF5CDF5CC906B6A
:1047BF00D7E0F5CBA3E0F5CA85CBCD85CACCE4F520
:1047CF00985387BF301906D29FD29E8002D29E4344
:1047DF008740C29FC2ACC298C29975B81075B71006
:1047EF00D2CAD29CD2AC12517EC2D9E5E92464F56B
:0D47FF00EB30D706E5F904F5FB2285F9FB48
:01480C002289
:0100220022BB
:01529B0022F0
:01529C0022EF
:1052100090637AE0B40118906382E0F54690638170
:10522000E0F547906380E0F54890637FE0F5492220
:1032D1009068DAE0FCA3E0FDA3E0FEA3E0FFEC4D83
:1032E1004E4F6007E54270037F0122854582854488
:1032F10083E07055F544F545200B077E257F0A12C2
:103301004259E4FF74742FF582E4346AF583E030A6
:10331100E30D74742FF582E4346AF5837407F00FBA
:10332100BF40E19068DAE0FCA3E0FDA3E0FEA3E08A
:10333100FFEC4D4E4F6006E4F5427F012285458248
:10334100854483E070037F0122854582854483A300
:10335100A3E0640160030233EC75350185443685D1
:103361004537E545241CF582E43544F583E06019D1
:1033710074202545F545E43544F544854582F583BA
:10338100E060030232EC7F0122301D2BE545241E53
:10339100F582E43544F583E030E01CE5452410FF77
:1033A100E43544F5838F8263A201906BB563A2017A
:1033B1007F0C1235BF801AE5452401FFE43544F541
:1033C100838F8263A201906BB563A2017F0C1235DA
:1033D100BFE545241EF582E43544F583E004F0851C
:1033E1004582854483E0F5380234C68545828544AB
:1033F10083A3A3E0FF64036003EF70320525532527
:103401000FE49069E3F0A3F0E5452401FFE43544BE
:10341100F5838F8263A201906BB563A2017F0C12C9
:1034210035BF854582854483E0F5380234C6AB3526
:10343100AA36A93790001C12302B700E7420254536
:10344100F545E43544F5440232ECE545241EF582A8
:10345100E43544F583E030E112E525600E74202562
:1034610045F545E43544F5440232EC854582854411
:1034710083A3E0906BB5F0854582854483A3A3E0E7
:10348100906BB6F0854582854483A3A3A3E0906B3E
:10349100B7F0E5452404F582E43544F583E0906B0B
:1034A100B8F0E5452405F582E43544F583E0906BF9
:1034B100B9F0E5452406F582E43544F583E0906BE7
:1034C100BAF0753806E4F53ED290C291C296D2990F
:1034D100200B0D7E257F187C6B7DB5AB38123F5ECE
:0234E1007F006A
:0134E30022C6
:103D2C00E54FC394404003E4F54FE534C394404061
:103D3C0003E4F53474982534F582E43468F583E0B3
:103D4C00FF30E17B74982534F582E43468F583EF19
:103D5C0054FDF0E4906476F0A3740DF090667BE073
:103D6C00906478F0A37419F0A37444F0A37439F040
:103D7C00E534C4135407FF906893E02F90647CF0F3
:103D8C00E534541F04A3F0A37408F0E53425E025B2
:103D9C00E024E3F582E43468F58363A20190647F48
:103DAC0063A2017F041235BF906483E549F0A3E55B
:103DBC0048F0A3E547F0A3E546F005347F012274F3
:103DCC0074254FF582E4346AF583E0FF30E16F74BB
:103DDC0074254FF582E4346AF583EF54FDF0E490DA
:103DEC006476F0A3740DF090667BE0906478F0A399
:103DFC007419F0A37448F0A37479F0E54F131313FE
:103E0C00541FFF906893E02F90647CF0E54F5407AB
:103E1C0025E025E02480A3F0A37408F0F5F0E54F2D
:103E2C00A42490F582E5F03466F58363A2019064D6
:103E3C007F63A2017F081235BF054F7F0122054F1A
:053E4C0005347F002297
:01529D0022EE
:10138D003000469080E8E0700F124EAF200B077EC4
:10139D00257F21124259C21E9080E8E0B40E1290B2
:1013AD0080037408F0200B077E257F2A124259C254
:1013BD001E9080E8E0B4060F201E0C200B077E2542
:1013CD007F35124259D21EC200201E0302148F20F7
:1013DD0090071245088F518003E4F551E5516047A0
:1013ED00200B0C7E257F4B7C6B7DDDFB123F5EE57C
:1013FD00E92410F5EB30D708E5F92428F5FB800634
:10140D00E5F92427F5FB906BDD63A201906BB563C5
:10141D00A201AF511235BF855138E4F53ED290C2CD
:10142D0091D21AC296D29920D903021C38C2D9E59D
:10143D00E92410F5EB30D708E5F92428F5FB8006F3
:10144D00E5F92427F5FBE539D394005003021C3848
:10145D00C291853943E4F539906AB563A201906B69
:10146D00DD63A201AF431235BFAF43124169300BAB
:10147D0003021C387E257F507C6B7DDDAB43123F14
:10148D005E227474253FF582E4346AF583E020E032
:10149D0002053FE53FC394404003E4F53F749825B2
:1014AD0024F582E43468F583E020E0020524E52488
:1014BD00C394404003E4F524123E51EF700302152E
:1014CD00B2E527B4010C852F46852E47852D48851D
:1014DD002C49E52A640F60030215B2906893E0FF72
:1014ED00652960030215B274982524F582E43468E9
:1014FD00F583E0FE30E05174982524F582E43468DC
:10150D00F583EE54FEF0752744752839E524C41390
:10151D005407FEEF2EF529E524541F04F52A752BEB
:10152D0008E52425E025E024E3F582E43468F5831D
:10153D007D2C7F041235B68549308548318547327B
:10154D00854633124F12805D7474253FF582E43465
:10155D006AF583E0FF30E04D7474253FF582E43485
:10156D006AF583EF54FEF0752748752879E53F132A
:10157D001313541FFF906893E02FF529E53F54078F
:10158D0025E025E02480F52A752B0875F008E53F48
:10159D00A42490F582E5F03466F5837D2C7F081246
:1015AD0035B6124F122002030216D5C202054AE5C6
:1015BD004AC39464406FE4F54AAF49AE48AD47ACB9
:1015CD0046FAF9F8EF2401F549EA3EF548E93DF50B
:1015DD0047E83CF546906890E0FEA3E0FFFBAA06C5
:1015ED00E4AF49AE48AD47AC46123105AC00AD0194
:1015FD00AE02AF03E4FBFAF9F8C31231A57026F57C
:10160D005174982551F582E43468F583E030E20E8B
:10161D0074982551F582E43468F5837403F005510F
:10162D00E551B440DCE54270529068DEE0FCA3E089
:10163D00FDA3E0FEA3E0FFE4FAF9F8EF2401FFEAD1
:10164D003EFEE93DFDE83CFC9068DE1231C9906834
:10165D00DAE0FCA3E0FDA3E0FEA3E0FFA3E0F8A326
:10166D00E0F9A3E0FAA3E0FBC31231A5400D7542EA
:10167D00019068DE1231D500000000906895E004FD
:10168D00F07006906894E004F0906896E0FEA3E098
:10169D00FFD3906895E09F906894E09E402AE4F017
:1016AD00A3F0F55174742551F582E4346AF583E0A5
:1016BD0030E20E74742551F582E4346AF5837403B7
:1016CD00F00551E551B440DC20D903021C38C2D9D4
:1016DD00E539D394005003021BD1C291853943E4FF
:1016ED00F539F50B7E6A7FB5AD431250CE200B0D4B
:1016FD007E257F557C6A7DB5AB43123F5E906A694E
:10170D00E0FF906A18E04F6010300B03021BD17E92
:10171D00257F5C124259021BD1854582854483A3E6
:10172D00E0FF906AB5E06F6010300B03021BD17EB5
:10173D00257F68124259021BD1854582854483A3BA
:10174D00A3E06401703D906AB6E0601A200B077E3D
:10175D00257F77124259E545241CF582E43544F581
:10176D0083E4F0021BD1D21B200B077E257F8F1245
:10177D004259E545241CF582E43544F5837401F0A6
:10178D00021BD1D21BE543C39406501DAB35AA36BF
:10179D00A93790001CE4123058300B03021BD17E88
:1017AD00257F95124259021BD1854582854483A31D
:1017BD00A3E0B4081CE545241FF582E43544F58308
:1017CD00E075F002A4FF9069E3E5F0F0A3EFF0807F
:1017DD001AE545241FF582E43544F583E075F004E0
:1017ED00A4FF9069E3E5F0F0A3EFF0E4F551E545D2
:1017FD00241CF582E43544F583E0FD7C0074017E04
:10180D0000A851088005C333CE33CED8F9FFEE5C66
:10181D00FEEF5D4E7003021BC5854582854483A393
:10182D00A3E064086003021A12301D41E55175F002
:10183D0003A424B6F582E4346AF583E0F552E4F5A9
:10184D003AE552543FF53BE55175F003A424B8F544
:10185D0082E4346AF583E0F53CE55175F003A42488
:10186D00B7F582E4346AF583E0F53D803FE55175C7
:10187D00F003A424B6F582E4346AF583E0F552E46E
:10188D00F53AE552543FF53BE55175F003A424B705
:10189D00F582E4346AF583E0F53CE55175F003A477
:1018AD0024B8F582E4346AF583E0F53DAF3DAE3CF6
:1018BD00AD3BAC3AE545241DF582E43544F583E0B6
:1018CD00F9F81231B68F3D8E3C8D3B8C3AE5523096
:1018DD00E71AE545241EF582E43544F583E030E052
:1018ED000BC3E4953DF53DE4953CF53CE55230E602
:1018FD001AE545241EF582E43544F583E030E60B08
:10190D00C3E4953DF53DE4953CF53C300C417E2519
:10191D007FA41242597559FF755A25755BA79069B9
:10192D00E3E0C313F55CA3E013F55DAF3DAE3CAD55
:10193D003BAC3A8F618E608D5F8C5E7B017A6979ED
:10194D00E5122D2B7E697FE57B057D0F1245E49019
:10195D0069E3E0FEA3E02490F58274663EF583E032
:10196D00653D60299069E3E0A3E0FF2490F5827462
:10197D00663EF583E53DF0EF7803CEC313CE13D865
:10198D00F92474F582746A3EF5837408F09069E465
:10199D00E004F070069069E3E004F09069E3E0FC88
:1019AD00A3E0FD2490F58274663CF583E0653C6010
:1019BD002A9069E3E0FEA3E0FF2490F58274663E71
:1019CD00F583E53CF0EF7803CEC313CE13D8F9249D
:1019DD0074F582746A3EF5837408F0EDAE047803F5
:1019ED00CEC313CE13D8F92474F582746A3EF583F1
:1019FD00E04404F09069E4E004F070069069E3E0DF
:101A0D0004F0021BC5201D03021AF0E55125E02547
:101A1D00E024B8F582E4346AF583E0FF9069E4E0F0
:101A2D0024E3F582E43468F583EFF09069E4E00493
:101A3D00F070069069E3E004F0E55125E025E0241F
:101A4D00B9F582E4346AF583E0FF9069E4E024E3BC
:101A5D00F582E43468F583EFF09069E4E004F0700A
:101A6D00069069E3E004F0E55125E025E024B6F5A4
:101A7D0082E4346AF583E0FF9069E4E024E3F582C3
:101A8D00E43468F583EFF09069E3E0FEA3E07802BB
:101A9D00CEC313CE13D8F92498F58274683EF5831E
:101AAD00E04404F09069E4E004F070069069E3E02E
:101ABD0004F0E55125E025E024B7F582E4346AF51C
:101ACD0083E0FF9069E4E024E3F582E43468F58374
:101ADD00EFF09069E4E004F070069069E3E004F043
:101AED00021BC5E55125E025E024B9F582E4346AF1
:101AFD00F583E0FF9069E4E024E3F582E43468F5D2
:101B0D0083EFF09069E4E004F070069069E3E0047F
:101B1D00F0E55125E025E024B8F582E4346AF5833B
:101B2D00E0FF9069E4E024E3F582E43468F583EFA7
:101B3D00F09069E4E004F070069069E3E004F0E5EC
:101B4D005125E025E024B7F582E4346AF583E0FF02
:101B5D009069E4E024E3F582E43468F583EFF090D6
:101B6D0069E3E0FEA3E07802CEC313CE13D8F924C7
:101B7D0098F58274683EF583E04404F09069E4E0E2
:101B8D0004F070069069E3E004F0E55125E025E0EE
:101B9D0024B6F582E4346AF583E0FF9069E4E0242D
:101BAD00E3F582E43468F583EFF09069E4E004F046
:101BBD0070069069E3E004F00551E551C3940450BB
:101BCD00030217FB201B0DAB35AA36A93790001C5D
:101BDD00E4123058E538600FE542600B742025455E
:101BED00F545E43544F544E5E924E8F5EB30D7084F
:101BFD00E5F92404F5FB8006E5F92403F5FB123223
:101C0D00D1EF7027854582854483A3A3E0B40319E2
:101C1D00E5E924F4F5EB30D708E5F92402F5FB806E
:0B1C2D0005E5F904F5FBD21B22C21BE9
:011C38002289
:03001E007F00223E
:10493B00021C39E493A3F8E493A34003F68001F23D
:10494B0008DFF48029E493A3F85407240CC8C3337D
:10495B00C4540F4420C8834004F456800146F6DF4C
:10496B00E4800B0102040810204080905294E47EF6
:10497B00019360BCA3FF543F30E509541FFEE49341
:10498B00A360010ECF54C025E060A840B8E493A308
:10499B00FAE493A3F8E493A3C8C582C8CAC583CA33
:1049AB00F0A3C8C582C8CAC583CADFE9DEE780BEEB
:01529A000013
:10302B00BB010CE58229F582E5833AF583E022505A
:10303B0006E92582F8E622BBFE06E92582F8E222A4
:0D304B00E58229F582E5833AF583E49322BE
:10305800F8BB010DE58229F582E5833AF583E8F0AE
:10306800225006E92582C8F622BBFE05E92582C85A
:02307800F22242
:10307A00E88FF0A4CC8BF0A42CFCE98EF0A42CFCF5
:10308A008AF0EDA42CFCEA8EF0A4CDA8F08BF0A473
:10309A002DCC3825F0FDE98FF0A42CCD35F0FCEBD2
:1030AA008EF0A4FEA9F0EB8FF0A4CFC5F02ECD3997
:0F30BA00FEE43CFCEAA42DCE35F0FDE43CFC2204
:1030C90075F008758200EF2FFFEE33FECD33CDCCBE
:1030D90033CCC58233C5829BED9AEC99E582984041
:1030E9000CF582EE9BFEED9AFDEC99FC0FD5F0D61E
:1030F900E4CEFBE4CDFAE4CCF9A88222B800C1B948
:103109000059BA002DEC8BF084CFCECDFCE5F0CB85
:10311900F97818EF2FFFEE33FEED33FDEC33FCEBBE
:1031290033FB10D703994004EB99FB0FD8E5E4F979
:10313900FA227818EF2FFFEE33FEED33FDEC33FC66
:10314900C933C910D7059BE99A4007EC9BFCE99A5A
:10315900F90FD8E0E4C9FAE4CCFB2275F010EF2F9F
:10316900FFEE33FEED33FDCC33CCC833C810D7079F
:103179009BEC9AE899400AED9BFDEC9AFCE899F8DA
:0E3189000FD5F0DAE4CDFBE4CCFAE4C8F9226D
:0E319700C3E49FFFE49EFEE49DFDE49CFC2249
:1031A500EB9FF5F0EA9E42F0E99D42F0E89C45F080
:0131B50022F7
:1031B600E8600FECC313FCED13FDEE13FEEF13FFF7
:0331C600D8F1221B
:0C31C900ECF0A3EDF0A3EEF0A3EFF02279
:1031D500A8828583F0D083D0821231EC1231EC12B3
:1031E50031EC1231ECE473E493A3C583C5F0C583D8
:1031F500C8C582C8F0A3C583C5F0C583C8C582C844
:0132050022A6
:10320600D083D082F8E4937012740193700DA3A357
:1032160093F8740193F5828883E47374029368606B
:06322600EFA3A3A380DF6B
:102CCF00E5652459F8E605652278563017027859DC
:102CDF00E475F00112325702322C2010EB7F2ED206
:102CEF00108018EF540F2490D43440D4FF30140BBD
:102CFF00EF24BFB41A0050032461FFE5666002158C
:102D0F00660569E5697002056830170D7856E47538
:102D1F00F001123257EF0232450250857403D21779
:102D2F008003E4C217F5658B568A578958E4F56618
:102D3F00F568F569E56660077F20122D0A80F57545
:102D4F0067FFC211C210C212C213C215C216C21837
:102D5F00122CD8FF700D3017057F00122D1BAF6995
:102D6F00AE6822B4255FC2D5C214122CD8FF24D06E
:102D7F00B40A00501A75F00A786630D50508B6FF08
:102D8F000106C6A426F620D5047002D21380D924DA
:102D9F00CFB41A00EF5004C2E5D214022F1BD21188
:102DAF0080C6D21080C0D21280BCD2D580BAD215C4
:102DBF0080B47F20122D0A2012077401B5660040DF
:102DCF00F1122CCFFF122D0A022D43D218D21680EA
:102DDF0095122CCFFB122CCFFA122CCFF94A4B7035
:102DEF000679EC7A2F7BFF20122EE566602A7E0093
:102DFF008E8275830012302B60060EEE656770F0C1
:102E0F00C2D5EBC0E0EAC0E0E9C0E0EE122F62D01D
:102E1F00E0F9D0E0FAD0E0FB12322CFF60AAEBC051
:102E2F00E0EAC0E0E9C0E0122D0AD0E02401F9D0B9
:102E3F00E03400FAD0E0FBE5670460DCD567D980A9
:102E4F00877BFF7A2F795ED212809C79108002796E
:102E5F0008C216C2188008D2D5790A8004790AC22E
:102E6F00D5E567047002F567E4FAFDFEFF122CCF7B
:102E7F00FC7B08201113122CCFFD7B1030100A128F
:102E8F002CCFFE122CCFFF7B20EC3382D592D55066
:102E9F0013C3E43010069FFFE49EFEE42011039D50
:102EAF00FDE49CFCE4CBF8C211EC700CCFCECDCC82
:102EBF00E824F8F870F38017C3EF33FFEE33FEED1D
:102ECF0033FDEC33FCEB33FB994002FB0FD8E9EBFE
:102EDF00301105F8D0E0C448B211C0E00AEC4D4EF5
:102EEF004F78207B0070C2EAB5670040BCC0E0128B
:102EFF002F64D0F0D0E0201104C4C0E0C4B211C0E0
:102F0F00F0122CF3D0F0D5F0EB022D431232062D38
:102F1F00E0532E5A582DB14C2DAD422E5E4F2E66DA
:0F2F2F00442E66492DC6432E6C552E50462E500B
:102F3E00452E5047300C502DB52D2DB92E2DDC2B96
:102F4E002DBD232DDA202FF52A2D754800002DD406
:102F5E003F3F3F00790AA2D5201314301509B9104E
:102F6E00020404B9080104A2D5201602500104205F
:102F7E0012689212B566005034C0E07F20301319EB
:102F8E007F30A21272167215500F122FBBC212C2D0
:102F9E0016C215C2187F30800F301503E9C0E0123B
:102FAE002D0A301503D0E0F9D0E0B566CC301517F8
:102FBE007F30B9100C122D0A7F583014077F78809D
:102FCE0003B90803122D0A3012057F2D022D0A7F38
:102FDE00202018F87F2B2016F322921280CF286E15
:102FEE00756C6C2900D211122CCF3011F8C21178E9
:102FFE006630D50108F6022D752D50434958122C16
:10300E00CF2403B405004001E490300793122CFB4B
:0D301E00743A122CFBD213756604022E5A70
:103890008B528A538954E4F55EF55DF55CF55BF572
:1038A00059F55AE556455745556012EBC0E0EAC058
:1038B000E0E9C0E0AB55AA56A957123267AB5205F2
:1038C00054E554AA537002055314F912322CF55FD3
:1038D000C394094007E55FD3940D40E1E55F6420A0
:1038E00060DBE55FB42D05435A038016E55FB42B1A
:1038F00005435A01800C74FF2554F55474FF355369
:10390000F553E55860046410703FAB52AA53A954B4
:1039100012322C64306009E558702E75580A8029DF
:1039200090000112302BFF64786004EFB458134309
:103930005A0175581074022554F554E43553F55363
:103940008007E5587003755808AB520554E554AA32
:10395000537002055314F912322CF55FC394614081
:103960000AE55FD3947A5003535FDF74D0255FF587
:103970005FC3940A400CE55F9411406D74F9255FB4
:10398000F55FE55FD395585060435A01855E6385C6
:103990005D62855C61855B60AF587E00E4FCFDABD9
:1039A0005EAA5DA95CA85B12307AC8ECC8C9EDC9F3
:1039B000CAEECACBEFCBE4FCFDFEEB255FF55EEE75
:1039C0003AF55DED39F55CEC38F55BAF5EAE5DADBB
:1039D0005CFCAB63AA62A961A860D31231A5500355
:1039E000023949435A04023949E55A20E003E48088
:1039F0002DE55645574555601EAB52E55424FFF959
:103A0000E55334FFFAEBC0E0EAC0E0E9C0E0AB55B3
:103A1000AA56A957123267E55A30E20774FFFFFE33
:103A2000FDFC22E55AAF5EAE5DAD5CAC5B30E10300
:043A300002319722A6
:10322C00BB010689828A83E0225002E722BBFE02A0
:09323C00E32289828A83E49322D3
:10324500BB010689828A83F0225002F722BBFE0168
:02325500F32262
:10325700FAE6FB0808E6F925F0F618E6CA3AF62278
:10326700BB011A89828A83D0F0D0E0F8D0E0F9D088
:10327700E0FAD0E0FBE8C0E0C0F00232BF5016E948
:10328700F8D083D082D0E0F9D0E0FAD0E0FBC0825A
:10329700C0830232B6BBFE16E9F8D083D082D0E0F5
:0F32A700F9D0E0FAD0E0FBC082C0830232C82227
:0932B600EBF608EAF608E9F6223D
:0932BF00EBF0A3EAF0A3E9F02210
:0932C800EBF208EAF208E9F22237
:00000001FF
